:020000040800F2
:100000005821012085010008C90100081D170008BA
:10001000C9010008C9010008C9010008000000006A
:10002000000000000000000000000000C9010008FE
:10003000C901000800000000C9010008C90100084A
:10004000C9010008C9010008C9010008C901000868
:10005000C9010008C9010008C9010008C901000858
:10006000C9010008C9010008C9010008C901000848
:10007000C9010008C9010008C9010008C901000838
:10008000C9010008C9010008C9010008C901000828
:10009000C9010008C9010008C9010008C901000818
:1000A000C9010008C9010008C9010008C901000808
:1000B000C9010008C9010008C9010008F9100008B9
:1000C00005110008111100081D110008C9010008E0
:1000D000C9010008C9010008C9010008C9010008D8
:1000E000C9010008C9010008C9010008C9010008C8
:1000F000C9010008C9010008C9010008C9010008B8
:10010000C9010008C9010008C9010008C9010008A7
:10011000C9010008C9010008C9010008C901000897
:10012000C9010008C9010008C9010008C901000887
:10013000C9010008C9010008C9010008C901000877
:10014000C9010008C9010008C9010008C901000867
:10015000C9010008C9010008C9010008C901000857
:100160002911000835110008C9010008C90100085B
:10017000C9010008C9010008C9010008C901000837
:04018000C9010008A9
:10018400002103E00A4B5B584350043109480A4BF1
:1001940042189A42F6D3094A02E0002342F8043B8B
:1001A400074B9A42F9D301F07DFE01F001FB704741
:1001B4003C380008000000203000002030000020FF
:1001C40054010120FEE7000037B5012002F092FA45
:1001D400002401902546E0B200F046F801AA08B9CF
:1001E40010551DE0135D042B0BDD174800F07EF95C
:1001F400019800F082F90120002102F06BFA00203E
:1002040020E00133DBB2042B135509D90F4800F069
:1002140055F9204600F071F90D4800F067F9012501
:100224000134042CD7D1019C3CB10A4800F046F9B2
:10023400204600F062F900F0D1F80120214602F0D6
:1002440049FA284603B030BDB0310008DC3100085B
:10025400E7310008F131000808B500F0A7FB80F091
:100264000100C0B208BD000008B5054B03EB001344
:100274005868198901F075FF003018BF012008BDC6
:100284003829000838B500242546E0B2FFF7ECFF12
:10029400A04001340543042CEDB2F6D1284638BD04
:1002A40073B50020014602F06DF80120002102F030
:1002B40069F80220002102F065F84FF48040012122
:1002C400104C02F0A3F904F14006684601F040FF27
:1002D40002238DF80530A37B60688DF80730002574
:1002E400A3688DF8045069461034009301F0F8FEB9
:1002F400B442EAD14FF48040294602F087F902B0B3
:1003040070BD00BF3829000810B5044608484021D4
:1003140002F0F6FA0028F9D00548214602F0ECFA7A
:100324000348402102F0ECFA0028F9D010BD00BFC8
:10033400001001402DE9F043DFF89890DFF8988031
:1003440087B01020012102F061F9484609210722F3
:1003540001F012FF07210A4606AD404601F00CFFEA
:100364004FF4007345F8183D00240226012748463F
:1003740029468DF806408DF807708DF804608DF8D5
:10038400056001F0ADFE80234046294600938DF8B8
:10039400046001F0A5FEADF80C40ADF80E40ADF8D8
:1003A4001040ADF8144004F1804404F58834084B3F
:1003B400029320460C2302A9ADF8123002F036FA5B
:1003C4002046394602F08CFA07B0BDE8F08300BF3E
:1003D40040420F0000000240000402402DE9F043B7
:1003E400334D83B02C6804F12E0323F0070300AFD0
:1003F400ADEB030D50238DF8003021238DF801302F
:1004040000238DF8023003238DF8033004F1210317
:100414005BBAADF80430274B04F127086E460DF1A2
:10042400060203F11C0153F8040B42F8040B8B423F
:10043400F9D11B78137004F12309224606F1230035
:100444001D4902F063FA31464A46002001F0D2FC0D
:1004540007F1080304F5927443F8040D186846F88C
:100464000900FE23B4FBF3F34344073323F00703EB
:10047400ADEB030D31464246684601F093FC044659
:100484005520FFF741FF6E466C44A64207D016F88C
:10049400010B552808BF0020FFF736FFF5E755206C
:1004A400FFF732FF00230C372B60BD46BDE8F08315
:1004B40030000020802900083400002010B5441EBC
:1004C40014F8012F7AB108490B68FF2B0BD80A2ABC
:1004D40002D1FFF783FFF3E70D2A1FBF581C5B18F7
:1004E40008601A71ECE710BD3000002008B5FFF772
:1004F400E5FFBDE80840FFF771BF1FB50C2201A955
:1005040001F0A8FC01A8FFF7D9FF05B05DF804FBD2
:10051400014608B5044802F080F90348022102F0BC
:100524007EF90028F9D008BD003800402DE9F047D5
:1005340007310733089E099F92464FEAD108DD0828
:1005440081460024B4420CD004EB0A03122000FBC1
:100554000380494638442A4602F0D8F90134A944B4
:10056400F0E7BDE8F087000008B54FF480400121B2
:1005740002F040F805484FF40071012201F0F7FD44
:100584000720BDE8084001F055BC00BF000402404C
:1005940008B5072001F04EFC4FF400710648002214
:1005A40001F0E5FD042001F045FC4FF480400021FA
:1005B400BDE8084002F01EB800040240F8B5074642
:1005C400FFF7D2FF8020FFF7A3FF0024661C30BA98
:1005D40090FAA0F0C0B2FFF79BFF122303FB047450
:1005E4000025605D00BA90FAA0F00135C0B2FFF7B3
:1005F4008FFF122DF5D10020FFF78AFFA82E344675
:10060400E4D10020FFF784FFBDE8F840FFF7C0BF46
:1006140010B5ADF6D83D02AC204600214FF43D6242
:1006240002F07FF91B238DE8180010214022692372
:100634000448FFF77BFF2046FFF7C0FF0DF6D83DC7
:1006440010BD00BF9D2900082DE9F043ADF6DC3D47
:1006540002AC00214FF43D620546204602F061F9E8
:100664002C238DE818002B48182120225C231C27FA
:10067400FFF75CFFBE460F23BB402B4023FA07F273
:10068400254B242101FB0233002202EBC20000F6B9
:10069400280013F802C020440021082907D00126AD
:1006A4008E4016EA0C0F14BF0126002603E09E18A4
:1006B400767806F0010686B101EB0E06F6B24FEA33
:1006C400D6094FF0010806F0070608FA06F610F8F6
:1006D400098046EA080600F8096001310929DCD1DD
:1006E4000232242AD1D10EF10B0EBEF1740FA7F100
:1006F4000407C0D10E238DE81800102190226D2329
:100704000648FFF713FF2046FFF758FF0DF6DC3DC0
:10071400BDE8F083172B0008272D0008672F000879
:1007240008B5FFF721FF0020FFF7F2FE0020FFF7D6
:10073400EFFE0020FFF7ECFEBDE80840FFF728BFFE
:10074400F0B5214B1A685E246043B0FBF1F4944287
:10075400ADF6DC3D34D002AD00214FF43D622846B5
:100764001C6002F0DEF81B238DE8280017481021D6
:1007740040226923FFF7DAFE08238DE82800144895
:1007840018216A226023FFF7D1FE002000F286714F
:1007940029440022A2420DD002F11903DBB2DF0882
:1007A400012603F0070306FA03F3CE5D3343CB556A
:1007B4000132EFE712306C28E8D12846FFF7FEFE3D
:1007C4000DF6DC3DF0BD00BF000000209D290008AF
:1007D4002B3000082DE9F843224E234CDFF88C908F
:1007E4004FF48040012101F005FF30460A21052223
:1007F40001F0C2FC04F10408052230460F2101F087
:10080400BBFC3046414601F06BFC01254FF40073FC
:100814000027304641466360A6F5E6362572A77286
:1008240001F05EFC414648462572A772656001F0FE
:1008340057FC304601F06EFF304604F10C0101F024
:10084400C1FF3046294601F0DCFF484629462A46C6
:1008540001F08DFC39464FF48040BDE8F84301F0C7
:10086400C9BE00BF00040240000000200000024096
:10087400F0B50746ADF2044D0E460C460025B919F5
:10088400B4F5806FA1EB040168460DD94FF4806282
:1008940000F0C4F8284669464FF4806201F0AAFAD1
:1008A400A4F580640546EAE7224600F0B7F8284636
:1008B4006946224601F09EFA0DF2044DF0BD08B5DA
:1008C400202001F0FDFD0028FAD108BD08B5022062
:1008D40001F0F6FD0028FAD00220BDE8084001F03E
:1008E400F9BD00B58DB0684601F073FD0023009397
:1008F4004FF4807368460A9335230B9301F09AFDF5
:10090400FFF7E4FFFFF7DBFF0DB05DF804FB000029
:1009140030B5022095B0012101F060FE0024224888
:100924000021204403220B460C3400F0C3F8482C69
:10093400F5D101A801F044FD10230024019301A87E
:10094400162305930294039404940694079401F0E7
:100954004FFD012001F092FDFFF7C3FF08A801F04D
:1009640038FD4FF44075662308A813930894129534
:1009740001F060FDFFF7AAFF08A801F02AFD992302
:1009840008A813930894129501F054FDFFF79EFFF5
:1009940042F6E06001F04EFAFFF7A3FF0220214681
:1009A40001F01CFE15B030BD8C30000830B50121BB
:1009B4008DB0022001F012FE022001F073FD6846A2
:1009C40001F007FD4FF0806300934FF040730493F0
:1009D4004FF4407368460A93AF230B9301F02AFD4A
:1009E400FFF774FF01F066FD054601F063FD044660
:1009F40001F060FD240244EA004040EA0504FFF7E8
:100A04005EFF0220002101F0E9FD0348231A584249
:100A140058410DB030BD00BFC225370070B5154632
:100A24008CB004460E460220012101F0D7FD681E59
:100A340001F038FD684601F0CCFC4FF08063009370
:100A44004FF040730493042305934FF440630993D8
:100A54004FF440730A934FF40053089368460B23F2
:100A64000B9301F0E7FC304601F014FD2544AC4241
:100A740004D001F01FFD04F8010BF8E7022001F097
:100A840029FDFFF71CFF0220002101F0A7FD0CB097
:100A940070BD0000024A136B43F0FF0313637047F9
:100AA40000380240024A136B23F0FF0313637047BC
:100AB4000038024013B504464068009002208DF8C7
:100AC40004008DF805208DF8061020682189A27A8B
:100AD4008DF8073001F050FB2068694601F000FBF7
:100AE40002B010BD02460068838823F4E0631B044F
:100AF4001B0C838003889BB243F400730380082398
:100B04000020517513751076704707B500230091C6
:100B140069468DF804308DF805308DF8073001F002
:100B2400DFFA03B05DF804FB10B50B4C342300FB73
:100B34000344236B7BB10A2001F081F96068A1684A
:100B4400FFF7E3FF20696169FFF7DFFF236B0120F3
:100B5400BDE81040184710BDD4300008027D082AB3
:100B640010B5044607D10268938823F4C0631B04BC
:100B74001B0C938084E0434B006803EB8203596BA6
:100B840001F0CAFB00287BD0237D072B72D8DFE855
:100B940003F0040B1921323B5A6E237A226803F0C6
:100BA400FE03138201232DE02268A37A1382637A61
:100BB4000BB1022326E093889BB243F480639380B5
:100BC40006231FE0226813889BB243F480731380CA
:100BD400032317E0237A226843F001031382E37AA4
:100BE400012B01BF138823F480631B041B0C08BF73
:100BF4001380042306E0226893889BB243F4806345
:100C04009380052323753BE023682269198A237B9B
:100C1400D154237BE27A0133DBB2591C9142237312
:100C240007D12268138823F480631B041B0C1380F0
:100C340026E0934224D12268938823F480631B0422
:100C44001B0C938013E0237B21692268CB5C138205
:100C5400237BE17A0133DBB29942237310D1938869
:100C640023F480631B041B0C93800723CAE72046EC
:100C7400012101E020460021BDE81040FFF732BF0A
:100C8400002010BDD43000082DE9F341184C342362
:100C940000FB0344236B43B300209847D4F804803B
:100CA400A668009600250127404669468DF8047021
:100CB4008DF805508DF8075001F012FAB1B22A46AA
:100CC400404601F054FA2669646900943046694646
:100CD4008DF804708DF805508DF8075001F000FA76
:100CE4003046A1B22A4601F042FA02B0BDE8F081D2
:100CF400D43000081C23104A434370B505460F4CFA
:100D0400D058D61801F04AFA342305FB03440021D5
:100D1400E06901F06FFC337923B92846BDE87040DF
:100D2400FFF7B2BF6068A168FFF7EFFE2069616951
:100D3400BDE87040FFF7E9BE34010020D43000085C
:100D44002DE9F04F344D1C2303FB005387B01B796E
:100D540007460BB9FFF7E8FE304B342407FB043495
:100D64000226D4F80490A389A26894F80EB00193E3
:100D74004FF001084FF0000A484602A902928DF88C
:100D84000C608DF80D608DF80E808DF80FA001F0C9
:100D9400A7F9019B484619465A4601F0EDF9D4F8E3
:100DA4001090238B626994F81AB00193484602A903
:100DB40002928DF80C608DF80D608DF80E808DF820
:100DC4000FA001F08DF9019B5A461946484601F0DF
:100DD400D3F94146E06901F00DFC02A801F076FA6E
:100DE4000F4A236A029393424FF48063ADF81230A2
:100DF4004FF01C0384BF626AADF80E2003FB07F4B6
:100E040002A9285901F0F8F92859012101F06CFAD6
:100E140007B0BDE8F08F00BF34010020D4300008D3
:100E2400A08601002DE9F341414C9846237F0546F5
:100E34000E4617461BB93F484FF4BD7103E020B17D
:100E44003C4840F27B1100F087FF23790BB9002066
:100E54006AE023681B8B9B0711D49DF82030E37252
:100E64000025099B277284F80A806672257325750C
:100E74002361E5822068012101F042FA1FE0FFF7B7
:100E840039FF2846FFF75CFF22682B48138B99072C
:100E9400E3D50138FAD1DAE7227E22B1019A511E54
:100EA4000191002AF8D100222276019A204902B346
:100EB4000A7D082A13D14D7D237D082B26D0236873
:100EC4001A8892B242F480721A809A8892B242F4DA
:100ED40040729A8001222276174A0192DEE7CA8A7A
:100EE400B2F57A7F05D20132CA82012000F0A7FF51
:100EF400E2E79A8822F4E0621204120C9A801A88BB
:100F040092B242F400721A8008230B7522680A4CCC
:100F1400138B9B0707D5013CFAD12046FFF7EAFE65
:100F24002046FFF70DFF284602B0BDE8F08100BF60
:100F3400340100203132000880841E00017D0368E2
:100F4400082906D19A8822F480721204120C9A801D
:100F540038E09A8A120541BF9A8A22F40062120488
:100F6400120C48BF9A829A8AD20541BF9A8A22F407
:100F740080721204120C48BF9A829A8A52051ED5B6
:100F84009A8A22F480621204120C04299A820AD1E9
:100F9400032202759A8822F4E0621204120C9A80E9
:100FA400002303760EE0012909D19A8822F4E06235
:100FB40012040021120C01759A80017602E00021CE
:100FC400FFF790BD0020704737B5124C124B2360D9
:100FD40008222275482200238DF8042001250C22C2
:100FE40001A88DF80520237123762373E37223610E
:100FF4008DF806308DF8075000F090FF492301A8C2
:101004008DF8043000F08AFF206801F0C7F82577D6
:1010140003B030BD34010020005C004013B50D4C1A
:10102400227F034622B90C484FF48C7100F094FEE1
:1010340038B1012200920848084A4FF48D7100F03B
:101044007FFE23790BB9FFF77BFE237901332371EC
:1010540002B010BD340100203132000846320008CD
:101064000C4A117F08B519B90B484FF4957103E088
:1010740020B1094840F22B1100F06EFE13793BB108
:10108400013BDBB213711BB9BDE80840FFF732BE68
:1010940008BD00BF340100203132000837B50D46C9
:1010A40014460093069B019301212A462346FFF729
:1010B400B9FE03B030BD07B500930123FFF7EEFF7F
:1010C40003B05DF804FB37B50D4614460093069B48
:1010D400019300212A462346FFF7A4FE03B030BD46
:1010E4001FB504AC04F8013D01230094FFF7EBFFA6
:1010F40004B010BD0148FFF731BD00BF340100202A
:101104000148FFF71BBF00BF340100200148FFF76F
:1011140025BD00BF500100200148FFF70FBF00BFED
:10112400500100200148FFF719BD00BF3401002021
:101134000148FFF703BF00BF3401002038B50C4657
:1011440005460020FFF76AFF234681212A46002036
:10115400FFF7B1FF04460020FFF782FF204638BDA9
:1011640038B50C4605460020FFF758FF234680217A
:101174002A460020FFF7B4FF04460020FFF770FF63
:10118400204638BD37B50D460DF107010446FFF77B
:10119400D5FF50B19DF807300121A9401943C9B2C8
:1011A40020468DF80710FFF7DBFF03B030BD0000C9
:1011B40013B590200DF10701FFF7C0FF044648B3B3
:1011C4009DF80740A4F111035C425C4114B3FF2174
:1011D4004220FFF7C5FFFF214120FFF7C1FF352063
:1011E4000DF10701FFF7AAFF044620B90B480C4A8A
:1011F400BE2100F0A5FD9DF80710352041F0030144
:101204008DF80710FFF7ACFF0A201E21FFF7A8FF97
:101214000028EBD0204602B010BD00BF7232000897
:101224009032000807B587200DF10701FFF786FF0C
:1012340018B19DF80700C0F3800003B05DF804FB0B
:1012440007B536200DF10701FFF778FF20B19DF8AF
:1012540007301B090B2B01D0002014E077200DF17F
:101264000701FFF76BFF0028F6D09DF8073003F065
:10127400100303F0FF0023B1FFF7D4FF80F0010057
:10128400C0B200F0010003B05DF804FB08B53620DD
:101294000121FFF777FF00B1FEE708BD07B5EF2195
:1012A4007420FFF75DFFFF217520FFF759FF0DF153
:1012B40007017720FFF742FF0DF107017820FFF7C0
:1012C4003DFF0A213920FFF74BFF35200421FFF7AA
:1012D40059FF00B1FEE703B05DF804FBB0F1006F05
:1012E40010B504460BD20C48FFF7E8F82046FFF788
:1012F40004F90A48FFF7FAF84FF0FF3010BD084B25
:10130400002053F8042BA24202D81A68944202D354
:1013140001300B28F5D110BDF0320008AF320008BF
:10132400283100082DE9F8430446174699460E462D
:10133400C1B3FFF7D3FF0546601E3044FFF7CEFF6D
:10134400002D804631DB00282FDB461B01361FB100
:10135400002031464A46B84700F022FE2C46444558
:101364001EDCF32000F032FE114B002133F8140090
:1013740000F064FE09280AD00E48FFF79FF82046C3
:10138400FFF7BBF8FFF72AF800F018FE0DE02FB1C5
:10139400C5F10100204431464A46B8470134DEE72E
:1013A40000F00CFE0120BDE8F8830020BDE8F883BE
:1013B40058310008C83200082DE9F0470E4615469A
:1013C4000746984600F0ECFDF32000F0FFFD4FEADD
:1013D400D51934463544AC42C6EB040A20D0B81BB8
:1013E400204414F8011B00F05FFE09280CD00F48BC
:1013F400FFF764F83846FFF780F8FEF7EFFF00F0D8
:10140400DDFD0020BDE8F087B8F1000FE3D01AF04D
:101414007F0FE0D14FEADA104946089AC047DAE76D
:1014240000F0CCFD0120BDE8F08700BFE0320008E9
:1014340008B545F2555000F07DFF042000F080FF10
:1014440040F6FF7000F082FF002000F073FF4FF4BD
:1014540080500121BDE8084000F096BD08B500F0B9
:1014640083FFBDE8084000F077BF08B57D2001F098
:1014740015F9003018BF012008BD4900FFF760B915
:101484002DE9F041012186B005460020FFF758F907
:10149400042000F0A3FB03A8294600F003FC03A8E2
:1014A40000F00FFC08B93C4814E03C480C35FFF749
:1014B4001DF804992846FFF7DBF904463848FEF77F
:1014C400FDFF2046FFF719F8FEF788FF059B9C42B5
:1014D40004D03448FFF70AF8012059E0049C32484C
:1014E400FFF704F82146314A31480023FFF71AFF79
:1014F4003048049FFEF7FAFF4FEA57080024BC4225
:1015040020D23E1BB6F5803F28BF4FF480362A48D0
:1015140061193246FFF782FA002304F10060009358
:1015240000F5804024493246FFF746FF18B92348A6
:10153400FEF7DCFF06E0344408EB54003946FFF7BD
:10154400FFF8DCE71E48FEF7B9FF0498FEF7D5FF65
:101554001C48FEF7B3FF1649049A002000F04AFC29
:1015640004461948FEF7AAFF0598FEF7C6FF174878
:10157400FEF7A4FF2046FEF7C0FFFEF72FFF059BF2
:101584009C4204D01248FEF7B1FF022000E0002084
:1015940006B0BDE8F08100BFF93200081733000837
:1015A400343300084A3300086D3300087F14000800
:1015B40000400008803300085101002093330008E4
:1015C4009E330008AC330008B5330008C833000864
:1015D400CE33000810B5022000F018FBD8B3042065
:1015E40000F014FB044670B11B48FEF77FFF042093
:1015F40000F000FB022000F0FDFA4FF40040BDE8CB
:10160400104000F0F7BA1548FEF770FF082000F00C
:10161400F1FA102000F0EEFA202000F0EBFA40205E
:1016240000F0E8FA2046FFF72BFF022807D1082034
:1016340000F0D4FA102000F0D1FA00F0A9FB042045
:1016440000F0D8FA022000F0D5FA4FF40040BDE8CB
:10165400104000F0C3BA10BD193400084F3400081C
:1016640010B52548FEF742FF4FF40010FFF708FFBE
:1016740010B102283AD809E0202000F0BBFA40203B
:1016840000F0B8FA802000F0A9FA2FE0082000F05A
:10169400A5FA102000F0A2FA202000F0B7FA20B931
:1016A4001648FEF723FF202007E0402000F0AEFAA2
:1016B40058B91348FEF71AFF402000F08FFA4FF490
:1016C400007000F08BFA00F063FB0E48FEF70EFF8B
:1016D400082000F08FFA102000F08CFA202000F08F
:1016E40089FA402000F086FA002400E00124042056
:1016F40000F080FA204610BD6A34000884340008E3
:10170400BD340008F634000808B50248FEF7EEFEC2
:1017140000F045FB303500081EF0040F0CBFEFF35A
:101724000880EFF30980FFF7EFBF704708B5012089
:10173400FEF79AFD08B900200FE00020FEF794FDA3
:101744000028F8D00220FEF78FFD0028F3D00320F4
:10175400FEF78AFD80F00100C0B200F0010008BD70
:101764001FB504461048FEF7C1FE01A90C2220460D
:1017740000F070FB01A8FEF7B9FE2046FEF764FFF7
:10178400FEF780FD094B20F0040018701C46FEF79C
:1017940079FD237800F0FB00834201D000F0F8FAD1
:1017A4000A2000F04CFBF2E7263500085101012025
:1017B40030B585B0FFF76EF94FF08050012100F08D
:1017C40019FF022000F0EAFD012807D1022000F0F1
:1017D400EFFDA548FEF78AFE00F0E1FA00214FF084
:1017E400805000F007FFFEF7A5FDA048FEF77EFE3F
:1017F4009F48FEF77BFE9F48FEF778FE9E48FEF763
:1018040075FE9E48FEF772FE9848FEF76FFEFFF7DE
:10181400DBFB9B48FEF76AFEFFF7CAFC9948FEF71C
:1018240065FE00F0FDF99848FEF760FE00F024FA2A
:1018340000210C2201A801F074F800F019FA01A9A2
:101844000C2200F007FB01A8FEF750FE8748FEF7C4
:101854004DFE8648FEF74AFE4FF4804000F0D6F96C
:1018640090B18A48FEF742FE4FF4804000F0C2F97E
:10187400082000F0BFF9102000F0BCF9202000F08F
:10188400B9F9402000F0B6F9FFF7DAFC38B1804826
:10189400FEF72CFE7F48FEF729FEFFF7FFFCFFF75B
:1018A40037F8FEF7FDFCFEF795FFFEF7B1FEFEF7F5
:1018B4008BFC08B1784803E0FEF7CEFC10B1774802
:1018C400FFF74EFF00F0C4F9802000F09FF918B133
:1018D400802000F08FF949E04FF4003000F096F9D1
:1018E40020B14FF4003000F085F95BE1FFF71EFFF3
:1018F40068B16B48FEF7FAFD41F28834FFF716FF32
:1019040078B1012000F09BFA013CF7D14AE1654B24
:101914000CCB013301D0013203D16348FEF7E6FD5D
:1019240040E1FFF7A2FD18B3FFF79FFD10B15F4838
:10193400FEF7DCFD4FF4007000F068F910B15C486C
:10194400FEF7D4FD4FF4007000F054F9102000F0BD
:101954005DF9D0B15748FEF7C9FD082000F04AF9F7
:10196400102000F047F9FFF77BFEF8B95248A7E7CB
:101974004FF4007000F04AF90028D5D1082000F097
:1019840039F9102000F036F90EE0082000F03EF995
:1019940020B14A48FEF7AAFD102003E04848FEF7AC
:1019A400A5FD082000F01AF9FFF714FE4FF40050CB
:1019B40000F02CF904464FF4805000F027F9400061
:1019C40040EA8400C4B24FF4006000F01FF92043E1
:1019D400C0B20728C3B20DD14FF4006000F00AF979
:1019E4004FF4805000F006F94FF4005000F002F973
:1019F400344865E70133DBB2023B4FF40060052B4A
:101A040011D8DFE803F00C1003100C1000F0F2F80A
:101A14004FF4805000F0EEF84FF4005003E000F073
:101A2400E9F84FF4805000F0D9F84FF4002000F0AA
:101A3400EDF8002851D04FF4002000F0DBF82248E4
:101A4400FEF754FD0024FFF7EDFB002840D0042CE2
:101A540003D11E48FEF74AFD00244FF4FA7000F04B
:101A6400EEF90134EFE700BF3B3500087C3700088E
:101A740048350008593500086A3500087B350008E8
:101A84008C35000897350008A3350008AC350008EC
:101A9400D93500080A360008014550FE024550FEBB
:101AA400293600080040000864360008773600082C
:101AB4008F360008AF360008034550FED7360008BD
:101AC400FD360008044550FE233700083737000868
:101AD4003648FEF70BFDFFF7D9FBFFF7A9FCFFF72C
:101AE400BDFCFEF7DFFF324B32485C681D68FEF731
:101AF400E5FC2046FEF701FD2F48FEF7DFFC00223F
:101B0400930003F1604303F5614301324FF0FF3169
:101B1400082AC3F88010C3F88011F1D1274B284A52
:101B2400196B0A401A635A6B22F0C0025A639A6B0B
:101B340022F003029A63196C224A0A401A64596C0F
:101B4400214A0A405A6400F0CBFC2048012100F0ED
:101B540069FD1E48002100F065FDF120012100F01F
:101B64006DFDF120002100F069FD0120014600F027
:101B740071FD0120002100F06DFD1548012100F0E8
:101B840075FD1348002100F071FD1248012100F099
:101B940079FD1048002100F075FD63B64FF0FF3E5B
:101BA400AD4620470C48FEF7A1FCDCE6523700089E
:101BB400004000086137000875370008003802400B
:101BC40000EF9FFF003619E8CC86E8FE0010E02203
:101BD400FFC9FEF6337F77047D37000810B504464D
:101BE400002000F087FD40EA04010020BDE8104019
:101BF40000F070BD10B50446002000F07BFD20EA23
:101C040004010020BDE8104000F064BD10B5044696
:101C1400002000F06FFD204214BF0120002010BD01
:101C240008B501214FF0805000F0E4FC012000F0E1
:101C3400A3FB4FF08050002100F0DCFC0120FFF7F3
:101C4400E5FF20B90121BDE8084000F043BD08BD0F
:101C540008B50648FEF732FC002000F04BFDFEF705
:101C64004CFCBDE80840FEF7B9BB00BF9C37000838
:101C7400022000F03FBD000008B5FFF7F9FF04495A
:101C8400884204D00220BDE8084000F023BD08BD0E
:101C94008BB8185808B50248FEF728FC00F078F80D
:101CA400A83700081FB504460C2201A8FEF7B6FEAB
:101CB40001AB03CB20601868A0602046616004B0CB
:101CC40010BD0068A0F10C03584258417047000051
:101CD40080B50646174610480D461C46FEF7EEFB37
:101CE4003846FEF7EBFB0D48FEF7E8FB3046FEF7FF
:101CF400E5FB0B48FEF7E2FB2846FEF7FEFB2CB1A2
:101D04000848FEF7DBFB2046FEF7D8FB0648FEF743
:101D1400EDFBFFF7BFFF00BFC537000856350008CD
:101D2400CE370008573500087C3700081FB506AACF
:101D340052F8044B039200921A462346FFF7C8FF59
:101D44000CB41FB506AA52F8043B03920092014A50
:101D5400FFF7BEFFD037000807B500230093724693
:101D6400014BFFF7E3FF00BFD7370008BFF34F8FE6
:101D74000549064BCA6802F4E0621343CB60BFF323
:101D84004F8F00BFFDE700BF00ED00E00400FA053F
:101D940008B5FEF7C5FC00F095FCFFF7E7FF08B5B2
:101DA400FFF7E4FFF0B5064600240120254603466C
:101DB40094421DD011F804C000F1010EBCF1000FD3
:101DC40003D17355774605460DE00133DBB2FF2B93
:101DD400774606F800C007D102F1FF3C644506D0FF
:101DE4007355871C7546012301343846E0E7704675
:101DF4007355F0BD30B5C9B1C0430A44914213D004
:101E040011F8013B0A4D83EA000404F00F0455F86D
:101E1400244084EA101080EA131303F00F0355F8EA
:101E2400233083EA1010E9E7C04330BD084630BDD3
:101E340070310008062358430138FDD1704710B5AE
:101E440004462CB14FF47A70FFF7F4FF013CF8E735
:101E540010BD00000A2A10B504DC1148BDE810408A
:101E6400FEF744BB0C46302304F8023B78234B7046
:101E74001C220F2393400340D340092B01D8303355
:101E840002E00F2B02D85733DBB200E02023043AE0
:101E940004F8013B131DECD100238B7210BD00BF6D
:101EA400233800081949D1F8883043F47003C1F885
:101EB4008830174B1A68002042F001021A609860BB
:101EC4001A6822F0847222F480321A60114A5A602D
:101ED4001A6822F480221A60D8601A6C0E4842F004
:101EE40080521A64026842F4404202609A689A601E
:101EF4009A689A609A6842F480529A604FF4C06279
:101F0400C3F800244FF000638B60704700ED00E0DD
:101F1400003802401030002400700040C27803787A
:101F240010B512B3164AD1684278C943C1F30221ED
:101F3400C1F10404E4B2A240D4B20F220A41817870
:101F44000A40224303F1604303F561431201D2B214
:101F540083F8002303780122590903F01F0302FACE
:101F640003F3084A42F8213010BD5A09012103F055
:101F74001F03994002F12003024A42F8231010BDC6
:101F840000ED00E000E100E0044B9A6809B1104361
:101F940001E022EA00009860704700BF002004E0DE
:101FA400044B1A69002ABFBF034A5A6002F18832FF
:101FB4005A607047003C024023016745024A136996
:101FC40043F0004313617047003C0240014BD8606A
:101FD400704700BF003C02400E4BDA68D20310D4B5
:101FE400DA68D1060FD4DA68D2050ED4DA6812F0B2
:101FF400E00F0CD1DB6813F0020F14BF0820092096
:102004007047012070470620704702207047072060
:10201400704700BF003C024007B509238DF8073024
:10202400FFF7DAFF8DF807009DF80730012BF7D092
:102034009DF8070003B05DF804FB000070B5064688
:1020440041B1012908D002290CBF4FF400754FF4A7
:10205400407503E00D4601E04FF48075FFF7DCFFA7
:1020640009281ED10F4C236923F44073236121698D
:1020740029432161236923F0F8032361236943F091
:1020840002031E432661236943F480332361FFF76F
:10209400C3FF236923F002032361236923F0F803B8
:1020A400236170BD003C024070B505460E46FFF743
:1020B400B3FF092811D1094C236923F44073236128
:1020C40023692361236943F0010323612E70FFF721
:1020D400A3FF236923F00103236170BD003C024088
:1020E400F0B50E6800220123934003EA060E9E45D4
:1020F4002AD1550003230468AB40DB431C40046031
:102104000C79076804FA05FC013C4CEA0707012C2A
:10211400076011D884684F791C4084608468AF409C
:1021240027438760446824EA0E0444608C79476836
:102134009440A4B23C434460C4682340C360CB7958
:10214400C468AB402343C3600132102ACBD1F0BD35
:102154004FF6FF7303600023037143718371C371EE
:1021640070470369194214BF0120002070470AB167
:10217400018370474183704701F00703C90800EBEE
:10218400810010B59B00046A0F21994024EA0101E3
:102194000162016A9A401143016210BD08B5134BF4
:1021A400984207D14FF40010012100F05FFA4FF478
:1021B400001014E00E4B984207D14FF48000012127
:1021C40000F054FA4FF4800009E00A4B98420BD116
:1021D4004FF40000012100F049FA4FF400000021FF
:1021E400BDE8084000F042BA08BD00BF00540040FA
:1021F40000580040005C00407FB5868826F03F060A
:102204000446360468460D46360C00F085F9029AF9
:102214002C48B2FBF0F081B20E43A68023882A4EEC
:1022240023F001031B041B0C23802B68B3420AD840
:102234005B000131B2FBF3F39BB2032B89B298BF6D
:102244000423218423E0EE884BF6FF718E421BBFEA
:1022540019214B4303EB4303B2FBF3F315BF9BB2CA
:10226400B2FBF3F343F480439BB2C3F30B020AB90A
:1022740043F001034FF4967101FB00F24FF47A71BD
:1022840092FBF1F2013292B243F400432284A3831D
:1022940023886989AA889BB243F001032380238899
:1022A40023F4816323F002031B040A431B0C13432E
:1022B4009BB223802A89AB8913439BB2238104B048
:1022C40070BD00BF40420F00A086010041F2883378
:1022D4000360002383804BF6FF72038143814FF434
:1022E4008043C28083817047038819B19BB243F055
:1022F400010303E023F001031B041B0C038070475C
:10230400038819B19BB243F4806303E023F4806330
:102314001B041B0C03807047838A9AB2038B10B58D
:1023240042EA034321F07F4404EA0300431A58427B
:10233400584110BD014B1860704700BF0030004089
:10234400014B5860704700BF00300040014B98605B
:10235400704700BF00300040024B4AF6AA221A60C0
:10236400704700BF00300040024B4CF6CC421A606C
:10237400704700BF00300040014B1860704700BF39
:1023840020000E4210B9034B19607047024B1960CC
:10239400704700BFA0000E429C000E42034B5B68D6
:1023A400184214BF01200020704700BF0070004095
:1023B400024A136843EA80001060704700700040CE
:1023C4000023036043608360C360036143618361EE
:1023D4007047002343608360C3600360036143610B
:1023E4008361C361036243628362C3627047000016
:1023F4000E4903680A6810B544691C4383691C4389
:1024040022F07F4323F030034268234343EA02630C
:102414000B60C36882684C681A43054B234013431E
:10242400026943EA02434B6010BD00BF001000A0E4
:10243400FEF7E0FF90E80C001A4383680D491A4345
:10244400C3681A4303691A4383691A43C3691A4365
:10245400036A1A43436A1A43836A1A43C36A10B568
:102464001A434C69044B23401343426943EA8243B1
:102474004B6110BD001000A000008090044B1A684E
:1024840010B142F0010201E022F001021A6070472B
:10249400001000A0024B9A68920658BF98617047DA
:1024A400001000A0024B9A68920658BF186170474A
:1024B400001000A0014B1878704700BF201000A046
:1024C400034B9B68184214BF01200020704700BFD3
:1024D400001000A0014BD860704700BF001000A09E
:1024E4000B4B1A68002142F001021A6099601A68C5
:1024F40022F0A85222F410221A60064A5A601A687E
:1025040022F480221A60D960C3F88C10704700BF8F
:1025140000380240103000242C4B9A6802F00C0260
:1025240010B50C2A38D8DFE802F0373737370737C9
:102534003737093737371E00254B2EE05968234AB1
:102544005B6811F4800F03F03F03516814BF204A05
:10255400204AB2FBF3F31D4A5268C1F388114B437E
:10256400C2F3014213E05968184A5B6811F4800F02
:1025740003F03F03516814BF154A164AB2FBF3F344
:10258400124A5268C1F388114B43C2F302720132FA
:102594005200B3FBF2F300E00E4B0C4A0360936865
:1025A4000D49C3F30313CC5C0368E34043609468B0
:1025B400C4F382240C5D23FA04F484609268C2F3A9
:1025C40042328A5CD340C36010BD00BF0038024071
:1025D40000127A000024F4001E000020044B9A6BC1
:1025E40009B1104301E022EA00009863704700BF7C
:1025F40000380240044B1A6C09B1104301E022EA8E
:1026040000001864704700BF00380240044B5A6C45
:1026140009B1104301E022EA00005864704700BF8A
:1026240000380240044B1A6909B1104301E022EA60
:1026340000001861704700BF00380240044B5A691B
:1026440009B1104301E022EA00005861704700BF5D
:1026540000380240044B9A6909B1104301E022EAB0
:1026640000009861704700BF00380240044B1A6AAA
:1026740009B1104301E022EA00001862704700BF6C
:1026840000380240044B5A6A09B1104301E022EABF
:1026940000005862704700BF003802404209012A16
:1026A400074B01D11B6803E0022A0CBF1B6F5B6F51
:1026B40000F01F0023FA00F000F00100704700BF93
:1026C40000380240024A536F43F0807353677047E7
:1026D4000038024082B000230193054B0193019B13
:1026E40003EB80000190019B196002B0704700BFAA
:1026F4005028004082B000230193054B0193019BB5
:1027040003EB80000190019B186802B0704700BF82
:102714005028004008B5254B984207D14FF480500B
:102724000121FFF7AFFF4FF4805039E0204B98426E
:1027340007D14FF480400121FFF798FF4FF4804008
:1027440009E01C4B98420BD14FF400400121FFF7E4
:102754008DFF4FF400400021BDE80840FFF786BF1D
:10276400154B984207D14FF400500121FFF78AFF1F
:102774004FF4005014E0114B984207D14FF48010ED
:102784000121FFF77FFF4FF4801009E00C4B9842C2
:102794000BD14FF400100121FFF774FF4FF4001028
:1027A4000021BDE80840FFF76DBF08BD00300140BF
:1027B40000380040003C004000340140005001401B
:1027C4000054014003884A8810B503F441540B882F
:1027D40013438A881343CA8813430A8913434A89D3
:1027E40013438A891343CA89134323439BB2038047
:1027F400838B23F400631B041B0C83830B8A0382E7
:1028040010BD038819B19BB243F0400303E023F0E9
:1028140040031B041B0C03807047818170470389AC
:10282400194214BF01200020704700007FB5038ABD
:10283400CA889BB223F440531343038283890E4610
:102844009BB223F4B053098923F00C02B3880B43E1
:1028540071890B439BB213438381838AB2899BB2F0
:1028640023F440731343838204466846FFF754FEFF
:102874001A4B9C4203D003F580639C4201D1039D13
:1028840000E0029DA38931681BB2002B4FF01902AE
:1028940002FB05F2B4BF4D008D00B2FBF5F5A28931
:1028A4006426B5FBF6F00001010912B2002A06FB0A
:1028B4001153ADBF1A01D90032313232B5BFB1FB69
:1028C400F6F2B2FBF6F302F0070203F00F03B4BF13
:1028D4001043184380B2208104B070BD0010014041
:1028E400838919B19BB243F4005303E023F40053EA
:1028F4001B041B0C83817047C1F30801818070475E
:102904000388194214BF01200020704710B5431EEC
:102914000A44914204D011F8014B03F8014FF8E73F
:1029240010BD02440346934202D003F8011BFAE7A8
:10293400704700001D32000800080240002000001B
:10294400020D000022320008000C024004000000C6
:102954000302020025320008001C024001000000AE
:10296400070002002C320008001C02400200000094
:1029740007010200000000000000000001424F4F68
:10298400544C4F414445520000000000002A2A00E4
:1029940000000000000000000000000000006000D3
:1029A40000030018000000000000000060000003A5
:1029B4000018000000000000000060000003001880
:1029C4000000000000000000600000030018000088
:1029D4000000000000006000000300180000000078
:1029E400E003001F60F800C30718C0070000F80FD9
:1029F400C07F60FE03F31F18F01F00000C1860C0B6
:102A04006003061B30181830000006303080E101E6
:102A14000C0F60180C60000003601800E300180736
:102A2400C01806C0008001400C006200100380182A
:102A34000380008001C00C0066003003801903800D
:102A4400018001C0FCFF670030038019FFFF018093
:102A540001C0FCFF630030038019FFFF008001C048
:102A64000C006000300380190300008001C00C00DA
:102A74006000300380190300008001400C006200F4
:102A8400100380180380008003601800C300180638
:102A9400C01806C000800730308081010C0C60181B
:102AA4000C6000800D1860C0000306183038183020
:102AB4000080F90FC07F00FE03F01F70F01F00803C
:102AC400E103001F00F800C00760C0070080010098
:102AD4000000000000000000000000800100000071
:102AE4000000000000000000008001000000000061
:102AF4000000000000000080010000000000000051
:102B04000000000000800100000000000000000040
:102B1400000000000C00060000000060003000000F
:102B240018000300000000C00018000030800100FD
:102B340000000080010C000060C0000000000000E4
:102B440003060000C060000000000000060300004F
:102B540080310000000000008C010000001B000018
:102B640000000000D8000000000E0000000000007B
:102B740070000000000E0000000000007000000063
:102B8400001B000000000000D8000000803100009D
:102B9400000000008C010000C06000000000000084
:102BA4000603000060C000000000000003060000EF
:102BB4003080010000000080010C000018000300B8
:102BC400000000C0001800000C00060000000060B7
:102BD40000300000000000000000000000000000C1
:102BE40000000000000000000000000000000000E1
:102BF40000000000000000000000000000000000D1
:102C040000000000000000000000000000000000C0
:102C140000000000000000000000000000000000B0
:102C240000000000000000000000000000000000A0
:102C34000000000000000080FFFF01000000000011
:102C4400000000FEFFFF7F00000000000000E07FA6
:102C54000000FE07000000000000FE010000807F6D
:102C64000000000000801F00000000F801000000C8
:102C740000F00100000000800F000000007C000054
:102C8400000000003E000000000F000000000000F3
:102C9400F00000008003000000000000C0010000FC
:102CA400E0000000000000000007000070000000C9
:102CB40000000000000E00001800000000000000EA
:102CC400001800000C0000000000000000300000AC
:102CD4000600000000000000006000000300000087
:102CE4000000000000C0008001000000000000009F
:102CF400008001C00000000000000000000003602C
:102D04000000000000000000000006300000000089
:102D14000000000000000C10000000000000000093
:102D24000000087C00FE00FF01C701C701C701C7FE
:102D340001C701C701C701C701C701C701C701C74F
:102D440001FF01FE007C0038003C003E003E0038DC
:102D540000380038003800380038003800380038AF
:102D64000038003800FE00FE00FE007C00FE00FF7C
:102D740001C701C701C001C001E000F00078003CB8
:102D8400001E000E000F000700FF01FF01FF017C81
:102D940000FE00FF01C701C701C001C001F80078AF
:102DA40000F800C001C001C001C701C701FF01FE56
:102DB400007C00E000E000F000F000F800F800F80B
:102DC40000FC00EC00EE00E600FF01FF01FF01E063
:102DD40000E000E000E000FF00FF00FF0007000744
:102DE4000007007F00FF00FF01C701C001C001C749
:102DF40001C701C701FF01FE007C007C00FE00FF4B
:102E040001C701C701070007007700FF00FF01C7E2
:102E140001C701C701C701C701FF01FE007C00FF14
:102E240001FF01FF01E000E0007000700070003855
:102E3400003800380038001C001C001C001C001C5A
:102E4400001C007C00FE00FF01C701C701C701C7C9
:102E540001FE007C00FE00C701C701C701C701C70E
:102E640001FF01FE007C007C00FE00FF01C701C7DA
:102E740001C701C701C701FF01FE01DC01C001C098
:102E840001C701C701FF01FE007C00000000000033
:102E94000000007C00FE00FF01C701C701F001FC37
:102EA40001CE01C701C701E701FF01DF01CE010720
:102EB40000070007000700E700F701FF01CF01C783
:102EC40001C701C701C701C701C701CF01FF01F74E
:102ED40001E70000000000000000007C00FE00FF8D
:102EE40001C701C7010700070007000700C701C7A2
:102EF40001FF01FE007C00C001C001C001C001CE81
:102F040001DF01FF01E701C701C701C701C701C70D
:102F140001C701E701FF01DF01CE0100000000004D
:102F24000000007C00FE00FF01C701C701C701FFCC
:102F340001FF010700C701C701FF01FE007C00E09B
:102F440000F000F8003800FE00FE00FE00380038F3
:102F540000380038003800380038003800380038AD
:102F6400003800000006830100000000000000009B
:102F7400000000068301000000000C0000000000B7
:102F840000068301000000000C00000000D8783621
:102F94009B79C0E3D90C8C67DB3C1BF8FD7EBFFD3D
:102FA400E0F7FB1FC6EFFB7E1F98CD66B3CD6036FE
:102FB4009B19C66C18660398FD66B3FD60309B19B7
:102FC400C66F18660398FD66B3FD60309B19C36F26
:102FD400186603980D66B30D60369B19C3601866B6
:102FE40003F8FD7EBFFDECF79B19C36F187E03D871
:102FF40078369B79CCE399998167183C03180000D3
:103004000000000000800100000000180000000023
:103014000000000000000000001800000000000094
:1030240000000000000000FFFFFFFFFFFFFFFFFFA5
:10303400FFFFFF010000000000000000000080010D
:1030440000000000000000000000800100000000FB
:1030540000000000000080010000000000000000EB
:10306400000080010000000000000000000080015A
:103074000000000000000000000080FFFFFFFFFFD1
:10308400FFFFFFFFFFFFFF000004024040000000BD
:1030940006000A00000402400400000002000900C7
:1030A4000008024000020000090009000008024074
:1030B400000400000A0009000008024000010000AA
:1030C400080009000000024002000000010009009D
:1030D400005C004000000240000100000800040001
:1030E4000004024000010000080009000000800004
:1030F400801A06000040000048490000000000005B
:1031040000000000010003008200070084000700A3
:1031140001000300020003004000030080000700D8
:103124008400070000000008004000080080000838
:1031340000C00008000001080000020800000408A4
:10314400000006080000080800000A0800000C0837
:1031540000000E08000008001000180020002800DD
:1031640030003800400048005000580000000000C3
:103174006410B71DC8206E3BAC30D9269041DC7674
:10318400F4516B6B5861B24D3C7105502083B8ED1E
:1031940044930FF0E8A3D6D68CB361CBB0C2649B42
:1031A400D4D2D38678E20AA01CF2BDBD53747563F1
:1031B4006B20627574746F6E2072656769737465D1
:1031C4007220697320696E76616C69642C20636C6B
:1031D400656172696E672E00427574746F6E206942
:1031E400642000697320737475636B2100427574E5
:1031F400746F6E2077617320707573686564206FD7
:103204006E20626F6F742E20427574746F6E20632B
:103214006F756E7465723A20004261636B0055707D
:103224000053656C65637400446F776E002E2E2F17
:103234007372632F647269766572732F6932632EB9
:1032440063004932432064657669636520494420FC
:103254006F7574206F6620626F756E6473202564C9
:1032640020286D61783A20256429006F6E002E2E87
:103274002F7372632F647269766572732F706D6930
:10328400632F617333373031622E63004661696C9A
:10329400656420746F20737461727420504D4943C7
:1032A40020313230487A2050574D00206973206F06
:1032B4007574736964652073797374656D20666CC5
:1032C400617368006661696C656420746F2065725F
:1032D40061736520736563746F7220006661696C45
:1032E400656420746F207772697465206164647208
:1032F4006573732000496E76616C69642066697237
:103304006D77617265206465736372697074696F47
:103314006E2100436865636B73756D6D696E67201C
:103324006669726D77617265207570646174650099
:1033340043616C63756C6174656420636865636B79
:1033440073756D3A2000496E76616C696420666914
:10335400726D776172652043524320696E20535029
:103364004920666C617368210065726173655F6FE3
:103374006C645F6669726D776172650077726974F7
:10338400655F6E65775F6669726D77617265005718
:1033940065277265206465616400436865636B73C7
:1033A400756D6D696E6720002062797465730D0A0E
:1033B40000436865636B73756D202D2077616E74AF
:1033C4006564200020676F7420004F757220696E59
:1033D4007465726E616C20666C61736820636F6ED5
:1033E40074656E7473206172652062616420286361
:1033F4006865636B73756D206661696C656429210A
:103404002054686973206973207265616C6C79203B
:1034140062616421004F75722070726576696F7500
:1034240073206669726D776172652075706461746A
:1034340065206661696C65642C2061626F727469D1
:103444006E67207570646174652E004E6577206622
:1034540069726D7761726520697320617661696C48
:1034640061626C6521004C6F6164696E67207265EE
:10347400636F76657279206669726D776172650033
:103484004661696C656420746F206C6F616420729E
:1034940065636F76657279206669726D77617265AE
:1034A4002C20737472696B65206F6E652E205472C4
:1034B4007920616761696E2E004661696C656420DC
:1034C400746F206C6F6164207265636F76657279C6
:1034D400206669726D776172652C20737472696BF2
:1034E400652074776F2E2054727920616761696E4C
:1034F4002E004661696C656420746F206C6F616492
:10350400207265636F76657279206669726D776182
:1035140072652C20737472696B65207468726565BA
:103524002E205341442057415443480048415244BB
:10353400204641554C540065786974207374616E5B
:1035440064627900205F5F5F20205F20205F20207D
:103554005F202020002F205F5F3E3C5F3E7C207C6C
:103564007C207C5F5F005C5F5F205C7C207C7C2037
:103574007C7C202F202F003C5F5F5F2F7C5F7C7C56
:103584005F7C7C5F5C5F5C0069326320696E697498
:10359400656400706D696320696E697465640062B6
:1035A4006F6F7420626974004C6173742066697271
:1035B4006D7761726520626F6F7420776173207319
:1035C4007461626C653B20636C6561722073747214
:1035D400696B657300504D494320776F6B652066B6
:1035E400726F6D207374616E6462792064756520F6
:1035F400746F206368617267657220646973636FB6
:103604006E6E6563740050757474696E6720504DF6
:103614004943206261636B20696E746F2073746127
:103624006E64627900486F6C6420646F776E205515
:1036340050202B204241434B202B2053454C4543E3
:103644005420666F72203520736563732E20746F67
:1036540020666F7263652D626F6F7420505246004E
:103664004669726D77617265206973206572617352
:103674006564005761746368646F67206361757380
:103684006564206120726573657400536F66747796
:10369400617265206661696C75726520636175731A
:1036A40065642061207265736574004661696C65A8
:1036B4006420746F207374617274206669726D770C
:1036C4006172652C20737472696B6520746872650D
:1036D400652E004661696C656420746F20737461A3
:1036E4007274206669726D776172652C20737472CE
:1036F400696B652074776F2E004661696C65642080
:10370400746F207374617274206669726D7761726C
:10371400652C20737472696B65206F6E652E00537F
:10372400687574646F776E207265717565737465FE
:10373400642E0052656D6F766520636861726765FB
:103744007220746F2073687574646F776E005368A9
:10375400757474696E6720646F776E2E00426F6FA4
:1037640074696E67206669726D77617265204020A6
:10377400002E2E2E0D0A0D0A00466F7263652D620F
:103784006F6F74696E67207265636F7665727920F6
:103794006D6F64652E2E2E00426F6F742062697403
:1037A400733A2000536F66747761726520666169AD
:1037B4006C7572653B20726573657474696E6721FC
:1037C400004153534552543A20003A004153534563
:1037D4005254004153534552544E002A2A2A20572A
:1037E4005446200053544D33320053544D33322049
:1037F4007065726970686572616C206C696272616F
:103804007279207472697070656420616E206173CE
:10381400736572740043524F414B204F4F4D006902
:10382400746F612062756666657220746F6F2073B1
:083834006D616C6C00000000E6
:10383C00FFFFFFFF008400000202000000C0040133
:10384C000000000000000002100000000700000053
:10385C00000001020304010203040607080900002A
:04000005080001846A
:00000001FF
